:103600000C942A1B0C943C1B0C943C1B0C943C1BF0
:103610000C943C1B0C943C1B0C943C1B0C943C1BCE
:103620000C943C1B0C943C1B0C943C1B0C943C1BBE
:103630000C943C1B0C943C1B0C943C1B0C943C1BAE
:103640000C943C1B0C943C1B0C943C1B0C943C1B9E
:103650000C943C1B11241FBECFE5D4E0DEBFCDBFD0
:1036600013E0A0E6B0E001C01D92AC33B107E1F772
:103670000E94201E0C94E71E0C94001BE0E0F0E07A
:1036800009950895899A8A9AD19AD29A0895809133
:1036900030038F5F8093300390911502992321F4BA
:1036A00080FF04C0DA9803C0913009F4DA9A8A30B6
:1036B00068F010923003992311F010923B0380912F
:1036C0003B038A3018F48F5F80933B0308959091F9
:1036D000600080912D03981710F00AC0A8955D9B9B
:1036E000FDCFE92FF0E0EF5FFD4F80818CB901C085
:1036F00092989F5F9093600008953CB180912C0355
:10370000882309F050C008B600FE06C080911A0256
:10371000813011F410921A0280911A02882371F4F8
:103720003A32E9F588B7816088BF12BE10922B0348
:1037300030932A0381E080931A020895813079F54D
:1037400090912B039F5F90932B039D3810F0109264
:103750001A02E92FF0E0E859FE4F308320912A0346
:10376000230F20932A03933041F4832F8C5F80939F
:10377000FE018D3810F010921A028091FE01981708
:1037800071F4822F831B80932A03381741F48091B0
:103790001A02813021F480932C0310921A0288B708
:1037A000816088BF12BE0895809104028B5F809370
:1037B0002D03E1E0F2E090E08150282F30E02E0F61
:1037C0003F1F02C08191980FE217F307D9F790834A
:1037D00081E080936000929A83E397E00197F1F78C
:1037E00001C0A8955D9BFDCF809101028CB9089521
:1037F000EF92FF920F931F93CF93DF9320911C02C0
:1038000030911D0240911E0250911F0220933103FE
:103810003093320340933303509334038091160264
:1038200090911702A0911802B09119022817390738
:103830004A075B0789F1E0903503F0903603009169
:10384000370310913803CCE1D2E020E030E0C90129
:1038500063E070E00E94A31E4C81892B21F0842F2D
:103860008F5F821B03C0842F8250820FE80EF11CF1
:10387000011D111DF901EC59FF4F80832F5F3F4F50
:1038800021962038310519F7E0923503F09236037E
:103890000093370310933803DF91CF911F910F915D
:1038A000FF90EF900895CF93DF9310921B02109238
:1038B0006300C0E0D0E0CE010E94B71E90911B02D1
:1038C000980F90931B029091630098279093630048
:1038D0002196CB30D10579F7DF91CF910895CF9321
:1038E000DF9310921B0210926300C0E0D0E0CE0183
:1038F0000E94B71E60911B02680F60931B0290919B
:1039000063009827909363002196CB30D10579F717
:103910008EE090E00E94C51E8FE090E06091630011
:103920000E94C51EDF91CF910895A89582E090E096
:1039300060E00E94C51E84E090E060E070E00E94BC
:10394000D21E86E090E060E070E00E94D21E88E027
:1039500090E060E070E00E94D21E8AE090E06DEF9F
:103960000E94C51EA8950E946F1C0895FF920F9398
:103970001F93F09069011091000280916A018117F4
:1039800009F05AC100916C01013009F043C08091E7
:103990006D01813019F40093150207C010921502D1
:1039A000823019F48EEF80936C0190911502913062
:1039B00091F58AE28093010210930202F0920302D1
:1039C0008CE08093040290930502909306028DE0B0
:1039D00090E0909308028093070280E092E0909339
:1039E0000A028093090280912E0390912F039093F5
:1039F0000C0280930B028091390390913A039093CB
:103A00000E0280930D0280E890E090931002809364
:103A10000F0210C190E080916C018230B9F4809166
:103A20001502813099F41092150260916D01862F74
:103A300082508D3F10F090E009C0609300028AE050
:103A400090E00E94C51E0E946F1C91E080916C0165
:103A50008330A1F580911502813081F570916E015E
:103A600060E080916D01680F711D70932F0360936A
:103A70002E0388E090E00E94D21E80E090E06FEF7D
:103A80000E94C51E81E090E06FEF0E94C51E0E945B
:103A90006F1C109235031092360310923703109268
:103AA000380380E090E0A0E0BFEF8093160290938F
:103AB0001702A0931802B093190291E080916C0153
:103AC000853009F059C080911502813009F054C049
:103AD00080916D0190916E01A0916F01B091700184
:103AE00080931C0290931D02A0931E02B0931F02AC
:103AF00090E0E92FF0E0DF01A859BE4F1B968C91B2
:103B0000E45EFD4F84839F5F903899F70E94F81B15
:103B100020913103309132034091330350913403AB
:103B200020308BE1380780E0480780E0580710F02C
:103B300090E022C08091160290911702A091180285
:103B4000B091190282179307A407B50721F0CA01A3
:103B5000B9010E94841F8091310390913203A0919A
:103B60003303B09134038093160290931702A0930D
:103B70001802B093190291E080916C01893019F517
:103B8000809115028130F9F420916D0130916E0120
:103B900040916F01509170018091350390913603EF
:103BA000A0913703B0913803281739074A075B07FC
:103BB00011F090E008C080E090E061E00E94C51E36
:103BC0000E946F1C91E020916C012E3F11F58AE25A
:103BD0008093010210930202F092030284E080932A
:103BE0000402209305028DE08093060280912E034B
:103BF00090912F03909308028093070280E090E059
:103C00000E94B71E8130B1F0109208021092070294
:103C100011C08AE28093010210930202F092030223
:103C200083E08093040284E68093050200930602F9
:103C3000909307020E94D41B1F910F91FF9008954B
:103C40000F931F93A8952FE088E190E00FB6F894AA
:103C5000A89581BD0FBE21BD10BC87E189B988E15F
:103C60008AB90E94421B82E090E00E94B71E8F3FFB
:103C700011F40E94951C8EE090E00E94B71E182F50
:103C80008FE090E00E94B71E082F0E94531C809185
:103C90001B02811721F480916300801711F00E94AC
:103CA000951C84E090E00E94BF1E90933A0380939D
:103CB000390386E090E00E94BF1E909362008093DB
:103CC000610088E090E00E94BF1E90932F038093D4
:103CD0002E038AE090E00E94B71E8093000284E0E9
:103CE00083BF8BE08EBD80E09DE29BBD8ABD18E066
:103CF000A89508B604FE05C088B7806188BF0E94F9
:103D0000471B5F9B02C00E947D1B5E9B03C05E9AA7
:103D10000E94671B80912C03882321F00E94B61C0F
:103D200010922C0380913B038450843008F7109349
:103D30003B0380E090E00E94B71E8130C9F6E0E0CE
:103D4000F0E00995D5CFAA1BBB1B51E107C0AA1F04
:103D5000BB1FA617B70710F0A61BB70B881F991F2C
:103D60005A95A9F780959095BC01CD010895E199E8
:103D7000FECF9FBB8EBBE09A99278DB30895A8E133
:103D8000B0E042E050E00C94D91E262FE199FECF1E
:103D90009FBB8EBB2DBB0FB6F894E29AE19A0FBE83
:103DA000019608950E94C51E272F0C94C61EDC01A3
:103DB000CB01FC01E199FECF06C0FFBBEEBBE09A50
:103DC00031960DB20D9241505040B8F70895F894D5
:023DD000FFCF23
:103F0000E0E0FBE1099508950F931F93CF93DF93B2
:103F1000A895BFB7E199FECF83E0FB0180935700DE
:103F2000E89507B600FCFDCF04E610E0AB01A1E088
:103F3000E801398120E08881F901E80FF11DCF0106
:103F4000FA010C01A0935700E89511240E5F1F4F52
:103F50004E5F5F4FF0E0043E1F0751F785E0FB0125
:103F600080935700E89507B600FCFDCF81E1809370
:103F70005700E895BFBFDF91CF911F910F91089532
:0400000300003600C3
:00000001FF
